:020000040000FA
:0200000079285D
:020008006F295E
:1000100086110C288615000006111220330E1220BE
:100020001C200800B3000F308605F030330586042D
:1000300086140000861008008316F03086048312B0
:10004000861100000615861406088610B300861473
:1000500006088610B31B232806118316F030860687
:1000600083120800061100008611000086100F3070
:1000700062213030122005306221303012205521AB
:1000800030301220552120301220552128300820F0
:1000900008300820013008200630082008008316A8
:1000A000F0308604831286150000061586140608B3
:1000B0008610F039B300B30E861406088610F039A6
:1000C000B304B30E06118316F03086068312552151
:1000D0003308080075208A110A12B20A0319B10AFE
:1000E000003E031908000A206A2831088A003208F5
:1000F0008200031383129F01831606309F00803015
:1001000081001830850001308600FF3087000C1414
:1001100083120130900000308B000430850086018E
:1001200032200C3008200330B400023008200130A7
:10013000B1001A30B2006A20C03008206A2069215C
:100140006721023008206A20C03008206A20692117
:100150006721023008206A20C03008206A20692107
:100160006721B40B95280130082069210C30082044
:1001700050308B00B601A101A201A301A4013C30C3
:100180008F00B0308E006430A000B61385148B173A
:100190000511B61BD0288519D0280130B606B61730
:1001A0002008031DC92805158B1305140000051030
:1001B0000708A40085109921DE20BB28B50127304F
:1001C00084003618B6143508031DEF2802300820C5
:1001D00020300A20B50A20300A20B50AE32804306E
:1001E00035020319F92808303502031DFF28C030F5
:1001F00008202C30B61820300A20B50AE3280C302D
:10020000350203181429B61C0B290008303C203095
:1002100003190C29B61000080A20B50A840A0B300D
:1002200035020319B610E3280130B1005030B20096
:100230006A200800203446347234653471342E3418
:1002400043346F34003475346E347434653472342E
:1002500049344934203400342034203420342034CC
:100260005634653472342E340034203431342E3414
:1002700030343134203420342034003420342034DD
:100280006234793420346D342E347934003461345E
:100290006D3461346D346F3474346F342034003411
:1002A000203448347A34203400346330B70058297D
:1002B000B70B572908000A30B8005521B80B5D2943
:1002C00008006430B9005B21B90B632908000530D0
:1002D0006A290A30BA006121BA0B6B290800F200C2
:1002E000030E8301F0000A08F1008A018B187B29B4
:1002F0000C18842992298B10A30A031D9229A20AA3
:10030000031D9229A10A92290C103C308F00B030B5
:100310008E00A00320308506200B922948308F00E4
:10032000E5308E0071088A00700E8300F20E720EA6
:1003300009002F308400A621A621A621A621A621EE
:10034000A621A621A621A621A62108002030AF00C3
:10035000B0010310A40DA30DA20DA10DB00DF63038
:1003600030070318B0000318A40AAF0BA9298403AF
:0A03700030088000303080070800DC
:02400E00323F3F
:1042000043006F0070007900720069006700680069
:1042100074002000280043002900200032003000F4
:104220003100370020006200790020004D002E0090
:10423000590061006D0061006D006F0074006F0037
:00000001FF
